:020000040000FA
:020000009D2839
:08000800B4000308B5008312E7
:100010000B19192828158B1810280B1919282811C5
:10002000281E2B210C108B1035088300B40E340EC3
:1000300009000B1164002F088500B30AA9080319F1
:100040002428A9030319A814B00803193128300A79
:1000500003193328B10B14282030AF063008B10043
:100060001428AF12031DAF160130B1001428333429
:100070002D344334683461346E346E3465346C34FA
:100080002034523465346C34613479342034433450
:100090006F346E34743472346F346C346C34653451
:1000A00072342034313432344634363432343934D4
:1000B0002F3436343734353443346F347034793434
:1000C00072346934673468347434203428344334E7
:1000D0002934203450346534743465342034473442
:1000E0007234693466346634693474346834733411
:1000F000203432343034313430342D3432343034EE
:1001000031343134203468347434743470343A34D3
:100110002F342F34703469346334703472346F3454
:100120006A3465346334743473342E346F34723407
:1001300067342E3475346B342034831A162A073012
:100140009900850183169F010C308500FF239000E4
:100150006400143081000C14831290018F018E0111
:100160008C01203084008001840A60300406031D65
:10017000B3280130B100FF30AE0081010B110B1626
:100180000B178B168B17A0211830B0006E30A9000A
:10019000A810A81CC9280030B000A814D920E2205B
:1001A0008519B3013308963A031DCE28D921B3012E
:1001B000CE28A81C08002818AE1728102009AF0563
:1001C000B0010800281E08002C08AD06031D2812E7
:1001D000AD002B08AE06031D2812AE00281E080035
:1001E0000721A81AFA281321A81AFA281F21A81AE9
:1001F000FA280329281800292814AF062005AF047F
:100200000C30A900A8100330B00028120800A81272
:1002100021082C06031D080022082B06031D0800D8
:10022000A81601300800A81223082C06031D080098
:1002300024082B06031D0800A81602300800A81287
:1002400025082C06031D080026082B06031D0800A0
:10025000A816103008002A0803193E29FF3E03198A
:100260004629FF3E03195229FF3E03195829FF3E34
:1002700003196F29FF3E03197E297A29281D7A293F
:10028000922105197A290130AA0008008421281931
:100290007A29051D7A292B308400403080000230F5
:1002A000AA0008008421281D7A290330AA0008002A
:1002B0008B2128197A290230AA000314051903108A
:1002C000800C031C08002C30840603196B29840061
:1002D00010308000080099210430AA000800281975
:1002E0007A290310AB0CAC0CAC0C2C0C1F39AC00F5
:1002F0002816802999210530AA00080028197A2992
:1003000010100030AA0008001010FC308F00903050
:100310008E00101408001010FB308F0064308E0027
:10032000101408001010F5308F0088308E00101463
:1003300008001010D1308F0034308E0010140800E7
:1003400020308400B60183169B011C141A0880001B
:10035000B6079B0A840A0408283A031DA5298312BC
:10036000270836022702031908007830B0008519E3
:10037000B729D921080020308400A70183169C18D2
:10038000BF299B0100089A008312A70783161C153A
:100390008B1355309D00AA309D009C148B179C1820
:1003A000CF299B0A840A0408283A031DC229831214
:1003B0000800EC30AF053D30B0002F1405222B08AB
:1003C000A2002C08A100AF1405222B08A4002C08C1
:1003D000A3002F1605222B08A6002C08A500143018
:1003E000B000851D112A281EF1292812A81C012AF7
:1003F0000721A81AAF061321A81AAF061F21A81AB1
:10040000AF060C30A900A810F129281E052AEC30EF
:10041000AF05A8102830281AA9002812A81C0A2AFB
:1004200008002F081339A000BB210800831285168D
:040430006400172A23
:02400E008C3FE5
:1042000000000100000001000100010008000C0096
:00000001FF
